:020000040000FA
:06000000D1EF07F0120031
:06080000D1EF07F0120029
:06082A000100D60F0000E2
:0808300060000000240000003C
:08083800D9CFE6FFE1CFD9FFA3
:10084000040EE126DE6ADE6ADE6ADD6ADD52DD5212
:10085000FD0EDBCF00F0FE0EDBCF01F0026A036A73
:1008600001AE02D002680368D9CFE9FFDACFEAFF10
:10087000030EEB500318E8AE02D0033408D000504A
:10088000EE5C0150EE580250EE580350EE580FE265
:100890000C0EE66EB1EC07F0E552D9CFE9FFDACFE6
:1008A000EAFFEE2A000EEE22EE22EE22D1D7040E4F
:1008B000E15C02E2E16AE552E16EE552E7CFD9FF81
:1008C00012000F0EC16E070EB46E936A300E926E58
:1008D0000F0E946EF19E1200D9CFE6FFE1CFD9FF43
:1008E000020EE1268250020B01E0010E080DF3CF4B
:1008F00002F08250010B040DF3CF01F08050200B69
:1009000001E0010EE824006E8050100B01E0010EA2
:10091000002401240224DE6EDD6ADECF00F0DDCF8C
:1009200001F000C0F3FF01C0F4FF020EE15C03E23E
:1009300000D0E16AE552E16EE552E7CFD9FF12003F
:100940008092320EE66EDFEC07F0E5528084320EC4
:10095000E66EDFEC07F0E5528094320EE66EDFECD7
:1009600007F0E55212008082320EE66EDFEC07F0EF
:10097000E5528084320EE66EDFEC07F0E55280949B
:10098000320EE66EDFEC07F0E5521200380E816E93
:10099000D7DF320EE66EE66A4FDFE552E552010E12
:1009A000816ECEDF320EE66EE66A46DFE552E55234
:1009B0000D0E816EC5DF320EE66EE66A3DDFE55252
:1009C000E552060E816EBCDF320EE66EE66A34DF5B
:1009D000E552E5521200010E816EB2DF0A0EE66E9C
:1009E000E66A2ADFE552E5521200D9CFE6FFE1CFF1
:1009F000D9FF020E816EA4DF0A0EE66EE66A1CDFE6
:100A0000E552E552FD0EDBCFE6FFFE0EDB50280D72
:100A1000F350E552E724E76EFE0EE7CFDBFFFD0E55
:100A2000DB6AFE0EDB50F36EFD0EDBCFF4FFF350FE
:100A3000F45C0BE2140E816E83DF0A0EE66EDFECCF
:100A400007F0E552FD0EDB2AECD7E552E7CFD9FFE0
:100A50001200D9CFE6FFE1CFD9FFFE0EDB50816E49
:100A600082DF320EE66EDFEC07F0E552E552E7CFAB
:100A7000D9FF1200D9CFE6FFE1CFD9FFFD0EDBCFC2
:100A8000E9FFFE0EDBCFEAFFEF500EE0FD0EDBCFFD
:100A9000E9FFDB2AFE0EDBCFEAFF01E3DB2AEF50A2
:100AA000E66ED7DFE552EAD7E552E7CFD9FF12006D
:100AB0000201046B300E926EF00E936EEF0E006F1B
:100AC00000C281FF040E016F0151000821E20051B4
:100AD000FE0BE842006F00C281FF050EE66EE66A7B
:100AE000ABDEE552E5528150100B09E08150200B3E
:100AF00006E08150400B03E08150800B01E10AD8F1
:100B00000201040502E1055104D00105016FDCD7A3
:100B1000CFD71200F00E936E81CF03F202010315BE
:100B2000026F0F0E0015006F00510211006F81CF90
:100B300003F2F00E0315026FF00E025D01E0F7D72D
:100B4000936A06D806C205F20201010E046F120074
:100B50000201076B100E075D14E20751EA6A600F8D
:100B6000E96E000EEA22EF50005D08E10751EA6AE3
:100B7000700FE96E000EEA22EFCF06F20729076F29
:100B8000E9D706C281FF640EE66EE66A55DEE552DD
:100B9000E55212000201086B070E085D1DE288DFB6
:100BA0000201096F0851EA6A0A0FE96E020EEA2291
:100BB00009C2EFFF0851EA6A0A0FE96E020EEA2243
:100BC000EF50460802E108D004D009C2E6FF41DF39
:100BD000E5520201082BE0D70851EA6A0A0FE96ED4
:100BE000020EEA22EF6A12000201086B070E085D8E
:100BF00016E20851EA6A0A0FE96E020EEA22EF5085
:100C0000E66E27DFE55202010829EA6A0A0FE96E5B
:100C1000020EEA22EF5001E102D0082BE7D71200C2
:100C200050DEB4DED8DE010E00018225826F000E98
:100C30008321836F806B816B100E81AF02D0D890BF
:100C400003D0805D000E81591AE280518225F66E34
:100C500081518321F76E340EF6260D0EF72208001F
:100C6000F550E66E130E8025E96E020E8121EA6EC4
:100C7000E552E750EF6E802B000E8123DDD7E66A48
:100C8000E66AB3DEE552E5520001806B816B080E27
:100C900081AF02D0D89003D0805D000E81590FE261
:100CA000130E8025E96E020E8121EA6EEF50E66E8A
:100CB000D0DEE5520001802B000E8123E8D7E66AE2
:100CC000010EE66E92DEE552E552080E0001806FDD
:100CD000816B100E81AF02D0D89003D0805D000EE2
:100CE00081590FE2130E8025E96E020E8121EA6E12
:100CF000EF50E66EAEDEE5520001802B000E812340
:100D0000E8D7130EE66E010EE66E96DDE552E5526B
:100D1000100E0001F76A8225F66E8351F722340E19
:100D2000F6260D0EF7220800F55002E1826B836B68
:040D30007AD712005C
:0C0D34002E2E2E2E2E2E2E2E2E2E2E2E8B
:100D40002E2E2E2E50554E544F20464C4F54414E71
:100D5000544520532E412E2E2E53495354454D4178
:100D6000204D4943524F434F4E54524F4C41444FF4
:100D70005220424F4C5420313846323535302E2ED9
:100D80003230204D485A2E2E33324B204D454D4F98
:100D900052494120464C4153482E2E324B204D455E
:100DA0004D4F5249412052414D2E2E323536204270
:100DB0005954455320444520454550524F4D2E2E01
:100DC00053454E534F522044452054454D504552B3
:100DD00041545552412E2E52454C455641444F5296
:100DE0002044452031323720562E206120312041C9
:100DF0004D502E2E38204C4544532E2E34204D4934
:100E000043524F53574954434845532E2E5055454E
:100E100052544F2055534220434F4E2050524F477B
:100E200052414D41444F5220494E5445475241444E
:100E30004F2E2E50554552544F2053455249414C48
:100E40002052532D3233322E2E50554552544F538B
:100E50002050415241204C43442059205445434C9A
:100E600041444F2E2E534F4654574152452044453E
:100E7000204445534152524F4C4C4F2050524F4604
:100E80004553494F4E414C2C20494E434C555945F2
:100E900020434F4D50494C41444F5220414E5349FD
:100EA00020432E2E2E2E2E2E2E2E2E2E2E2E2E2E5B
:100EB0000000000000000000000000000000000032
:040EC000000000002E
:0C0EC4002A0EF66E080EF76E000EF86E97
:100ED00002010900F5502C6F0900F5502D6F03E158
:100EE0002C6701D03DD00900F550276F0900F5505F
:100EF000286F0900F550296F09000900F550E96EC7
:100F00000900F550EA6E090009000900F5502A6F42
:100F10000900F5502B6F09000900F6CF2EF2F7CF2C
:100F20002FF2F8CF30F227C2F6FF28C2F7FF29C20E
:100F3000F8FF02012A5302E12B5307E00900F550A4
:100F4000EE6E2A07F8E22B07F9D72EC2F6FF2FC262
:100F5000F7FF30C2F8FF02012C07000E2D5BBFD750
:020F600012007D
:0E0F6200FF0EE350066E480E01D04C0EE76EF7
:100F7000E72EFED7E76AE72EFED7062EF7D700004A
:020F800012005D
:0E0F8200000EF36E00EE00F0080E01D8120013
:100F9000EA6002D0EE6AFCD7F350E9601200EE6A14
:020FA000FCD77C
:0E0FA20012EE40F022EE40F0F86A059C62EC80
:0E0FB00007F0EAEC07F010EC06F0FBD7120099
:020FBE00FF0E24
:100FC000E350E84E1200000000D000D000D0E82E20
:040FD000FAD712003A
:020FD400120009
:0A0FD600EEEDEBE7DEDDDBD7BEBD7C
:100FE000BBB77E7D7B773031323334353637383995
:0A0FF0004142434445460000000062
:00000001FF
